:020000040000FA
:0200000063D1CA
:08000800F2B20CD0F2B412D0E8
:020010001100DD
:08001800076ED8CF06F0E0CF1F
:1000200005F072D0F292808EC3EC01F032C033F052
:1000300026941100F2940F0E89129212EC0E8A127D
:1000400093120850F92652D040D032D020D012D08E
:100050008A9E0F0E0914921AE00E09148009931A51
:1000600009BE939618B204D002A002D02FB0939488
:10007000086A49D08A9C0F0E0A14921AE00E0A14DC
:100080004009931A0ABC93960A0E086E3CD08A9ACD
:100090000F0E0B14921AE00E0B142009931A0BBAD0
:1000A000939618B202D026B89394080E086E2BD0FF
:1000B00089960F0E0C140809921AE00E0C14931A6C
:1000C0000CB69396060E086E1ED089940F0E0D1472
:1000D0000409921AE00E0D14931A0DB4939618B2F7
:1000E00002D026B69394040E086E0DD089900F0EA0
:1000F0000E140109921AE00E0E14931A0EB0939684
:10010000020E086E00D011009E92196619061A663A
:100110001A06332E03D080AE2684809E352E0CD056
:10012000C80E356E26B002D0269601D0268626B29D
:1001300002D0269801D02688152E0AD0020E156E00
:100140001650500B176E8050500B166E1762168E9D
:1001500005C0E0FF075006C0D8FF10001F1F1D1F7D
:0A0160001E1F1E1F1F1E1F1E1F0082
:100200006F6F6F066FAB6F8F6FC66FCD6FED6F0740
:100210006FEF6FCF066F060606AB068F06C606CDDC
:1002200006ED060706EF06CFAB6FAB06ABABAB8FA9
:10023000ABC6ABCDABEDAB07ABEFABCF8F6F8F06E4
:100240008FAB8F8F8FC68FCD8FED8F078FEF8FCFB7
:10025000C66FC606C6ABC68FC6C6C6CDC6EDC60738
:10026000C6EFC6CFCD6FCD06CDABCD8FCDC6CDCD34
:10027000CDEDCD07CDEFCDCFEC6FEC06ECABEC8F39
:10028000ECC6ECCDEDEDEC07ECEFECCF076F07061D
:1002900007AB078F07C607CD07ED070707EF07CFA7
:1002A000EF6FEF06EFABEF8FEFC6EFCDEFEDEF07A0
:1002B000EFEFEFCFC76FC706C7ABC78FC7C6C7CDB6
:1002C000C7EDC707C7EFCFCFD3507009D36E896A88
:1002D0007F0EC16E500E926E8A6A130E936E190EC7
:1002E000AF6EAC6A8CEC04F0A0EC04F00450AA0AE7
:1002F00002E08CEC04F0500E166E050E156E320EF8
:10030000326EC30ED56ED66ACA6ACC6A2B0ECA6E1E
:10031000D10ECB6ECA84F26A9D6AA06A9E6AC00E34
:10032000F06EC50EF16E9F6AD08E9D82F00EF26E59
:10033000900EAB6E1882CF0E0E6EE30E0D6ECD0ECC
:100340000C6EE80E0B6EAE0E0A6E6E0E096EFA0E95
:1003500082EC04F02C0E0E6E0D6A6F0E0C6E800E89
:100360000B6E060E0A6E096AFA0E82EC04F0189201
:1003700016A886EC03F016AC3AEC04F0EFEC01F0B2
:10038000C4EC04F0F5D718B2120018B412001B50D8
:10039000E2EC01F06F0E106202D003A0106A10C0F0
:1003A0000EF011C00DF01C50E2EC01F010C00CF08A
:1003B00011C00BF01D50E2EC01F010C00AF011C0AA
:1003C00009F01200106E102610C0F6FF020EF76E34
:1003D0000900F5CF10F00800F5CF11F01200ABA224
:1003E00005D0AB98AE50AE50AE50AB88ABA401D0A8
:1003F000AE50FDEC02F0FA0A5AE02150240A01E066
:10040000F8D7FDEC02F0236E470A51E1FDEC02F053
:10041000500A4DE1FDEC02F0520A4AE02150470A31
:1004200046E1FDEC02F0470A42E1FDEC02F0410A30
:100430003EE1FDEC02F02C0A3AE1FDEC02F0D00FB7
:100440000A0DFDEC02F0D00FF324276EFDEC02F054
:10045000D00F0A0DFDEC02F0D00FF324286EFDEC56
:1004600002F0D00F0A0DFDEC02F0D00FF324296E3C
:10047000246AFDEC02F02C0A0AE021502E0A04E165
:10048000FDEC02F0D00F246E010EF0EC02F0050E30
:10049000F0EC02F0FDEC02F0D00F0A0DFDEC02F0E2
:1004A000D00FF324256E01E102E0268283D01200F2
:1004B000FDEC02F04D0AFBE1FDEC02F0430AF7E12E
:1004C000FDEC02F02C0AF3E1FDEC02F0D00F0A0D76
:1004D000FDEC02F0D00FF324276EFDEC02F0D00FFC
:1004E0000A0DFDEC02F0D00FF324286EFDEC02F0B3
:1004F000D00F0A0DFDEC02F0D00FF324296E246A10
:10050000FDEC02F02C0A0AE021502E0A04E1FDEC79
:1005100002F0D00F246E010EF0EC02F0FDEC02F0C0
:10052000410AC5E1070EF0EC02F0FDEC02F0D00F3D
:100530000A0DFDEC02F0D00FF3242A6EFDEC02F060
:10054000D00F0A0DFDEC02F0D00FF3242B6EFDEC62
:1005500002F0D00F0A0DFDEC02F0D00FF3242C6E48
:10056000FDEC02F0FA0AD8B457EF02F021502A0A43
:10057000F7E123502D6EFDEC02F0D00F226E0A0E33
:10058000225C02E3070E225EFDEC02F0300E215EDB
:100590000A0E215C02E3070E215E223821102D187D
:1005A000D8A457EF02F026802C50206E2B501F6EDF
:1005B0002A501E6E27501B6E28501C6E29501D6E2F
:1005C000346A269E189400A003D01B2A4CEC03F03A
:1005D00011EC03F041EC03F002667BEC03F020D059
:1005E0002E6EFDEC02F0FA0AD8B4120021502C0A4B
:1005F000D8A4F7D72E2EF5D71200060E196E9EBA84
:1006000007D01966FCD7342A420E3460268EFA0CC5
:10061000AE50216E2A0AD8B412002150231A1200BB
:10062000120001B805D001501B264CEC03F012005B
:100630000F0E01141B5E1BAE21D0180E1B261E2EA2
:100640001DD01F2E08D00C0E1F6E200620AE03D02A
:10065000630E206E0AD0020E1F6207D0030E201414
:10066000D8B403D01C0E1E6E09D0010EF76E1FC049
:10067000F6FF5C0EF6260800F5CF1EF04CEC03F0FA
:1006800012001D2A3B0E1D6412001D6A1C2A3B0E1F
:100690001C6412001C6A1B2A2F900C0E1B602F80FA
:1006A000170E1B641200180E1B5E2F900C0E1B60A1
:1006B0002F801E2A020E1F6206D0030E2014D8B40B
:1006C00002D01C0E07D0010EF76E1FC0F6FF5C0EA5
:1006D000F62608001E50F55CD8B01200010E1E6E02
:1006E0001F2A0C0E1F641200010E1F6E202A640EBA
:1006F0001F60206A12001B6603D00C0E1B6E1200D6
:100700000C0E1B6412000C0E1B5E12001882CD0E24
:100710000E6EE90E0D6EE00E0C6E6E0E0B6EE30E9D
:100720000A6E096A19EC04F0AE0E0E6ECD0E0D6E57
:10073000E00E0C6E0B6A0A6A096A00501CEC04F0A9
:1007400027EC04F016A80BD016BCFAD7002A020E2C
:100750000060006A00501CEC04F01880F1D7E00E35
:100760000E6EAB0E0D6E0C6A0B6A0A6A096A19EC02
:1007700004F00F0E01141CEC04F027EC04F0000E42
:1007800001B8800E0B6E16A80CD016BCF6D7012A45
:10079000200E0160016A01500F0B1CEC04F0188060
:1007A000ECD7E40E0E6EAC0E0D6E2C0E0C6EA00E81
:1007B0000B6E0A6A096A19EC04F0180E02660C0E38
:1007C0001CEC04F027EC04F016A80DD016BCFAD7E8
:1007D000022A020E0260026A180E02660C0E1CEC5F
:1007E00004F01880EFD7680E0E6EE90E0D6EE70E5E
:1007F0000C6EAE0E0B6E0A6A096A19EC04F0035017
:100800001CEC04F027EC04F016A80BD016BCFAD7A9
:10081000032A020E0360036A03501CEC04F01880E4
:10082000F1D719EC04F0189218B092EC04F018907B
:10083000120016A8FED71200E2EC01F06F0E106253
:1008400001D0106A10C00AF011C009F012000AC0ED
:1008500013F009C014F00A6A096A0A0E82EC04F067
:1008600013C00AF014C009F016B01200140E82EC86
:1008700004F01200188226B00DD0670E0E6EAC0E7A
:100880000D6EAE0E0C6EE70E0B6EE00E0A6EE90EEC
:10089000096E21D0AE0E0E6EE70E0D6EE00E0C6EE0
:1008A000E90E0B6E0A6A096A16ACFED71E50E2EC1E
:1008B00001F010500E6E11500D6E1F50E2EC01F061
:1008C00010500C6E11500B6E2050E2EC01F01050E5
:1008D0000A6E1150096E640E82EC04F0FA0E82EC7E
:1008E00004F0CD0E0E6EE70E0D6EE00E0C6E0B6A70
:1008F0000A6A096A25501CEC04F0FA0E82EC04F036
:10090000189212001A6E169016AE03D0169E16801C
:1009100012001A66F9D7120000EE00F0EE6AEAA0A3
:10092000FDD71200AA0E046E306A050E316E00EE7D
:1009300000F0EE50ADEC04F0302A312EFAD7120060
:10094000306A050E316E00EE00F03050BEEC04F05F
:10095000EE6E302A312EF9D71200A6B2FED7A86E5D
:1009600030C0A9FFA69EA69CA684F29E550EA76E37
:10097000AA0EA76EA682F28EA6941200A96EA69E5B
:10098000A69CA680A850120026AE0DD01884670E33
:100990000E6EAC0E0D6EAE0E0C6EE70E0B6EE00E14
:1009A0000A6EE70E096E26A40CD0670E0E6EAC0E12
:1009B0000D6E060E0C6EE30E0B6EE30E0A6ECD0E80
:0409C000096E1200AA
:020000040030CA
:03000100080E1EC8
:020005008081F8
:0600080003C003E0034009
:00000001FF
